:020000040000FA
:040000000BEF16F0FC
:080008001BEF09F0D9CFE5FF61
:10001000E1CFD9FF00C0E5FF01C0E5FF02C0E5FF69
:1000200003C0E5FF04C0E5FF05C0E5FF06C0E5FF2E
:1000300007C0E5FF08C0E5FF09C0E5FF0AC0E5FF0E
:100040000BC0E5FF0CC0E5FF0DC0E5FF0EC0E5FFEE
:100050000FC0E5FF10C0E5FF11C0E5FF12C0E5FFCE
:1000600013C0E5FF14C0E5FF15C0E5FF16C0E5FFAE
:10007000020EDBCF00F0030EDBCF01F0040EDBCF6E
:1000800002F0050EDBCF03F0060EDBCF04F0070E07
:10009000DBCF05F00550E56E0450E56E0350E56ECC
:1000A000F7EC11F0066E030EE1260050090F076E03
:1000B000000E0120086E000E0220096E07C0E9FF45
:1000C00008C0F3FF0950B2EC15F00A6EF3CF0BF045
:1000D0000A500B10D8A444D00650AA0A24E00050BD
:1000E000050F0C6E000E01200D6E000E02200E6E2C
:1000F0000CC0E9FF0DC0F3FF0E50B2EC15F00F6E0F
:10010000F3CF10F00F2AD8B0102A0FC0E5FF10C0AF
:10011000F4FF0CC0E9FF0DC0F3FF0E5017EC16F012
:10012000F36AE86A7FD1000EE56E00C0E9FF01C006
:10013000F3FF025023EC16F000500B0F0C6E000E74
:1001400001200D6E000E02200E6E000EE56E000EF8
:10015000F46E0CC0E9FF0DC0F3FF0E5017EC16F063
:100160000050110F0C6E000E01200D6E000E0220CB
:100170000E6E0A500C240F6E0B500D20106EE86AA4
:100180000BBEE8680E20116E06C0E5FF0FC0E9FF48
:1001900010C0F3FF115023EC16F00A2AD8B00B2A36
:1001A0000AC0E5FF0BC0F4FF07C0E9FF08C0F3FF7A
:1001B000095017EC16F007C0E9FF08C0F3FF09501B
:1001C000B2EC15F00F6EF3CF10F000500B0F116E64
:1001D000000E0120126E000E0220136E11C0E9FF06
:1001E00012C0F3FF1350B2EC15F0146EF3CF15F0FC
:1001F000070E1426D8B0152A0B50800FF36E155039
:10020000800FF35C02E114500A5C13E200C0E9FFC6
:1002100001C0F3FF0250DCEC15F00A6E06500A260E
:100220000AC0E5FF00C0E9FF01C0F3FF025023EC64
:1002300016F01050800F800F02E1060E0F5C03E2F3
:10024000F36A010EEFD00F50060A02E1105001E0F0
:1002500037D006C00AF00B6A0AC0E5FF0BC0F4FFF6
:1002600011C0E9FF12C0F3FF135017EC16F00B504A
:10027000800F800F02E1090E0A5C22E30050030F99
:100280000A6E000E01200B6E000E0220146E0AC0D2
:10029000E9FF0BC0F3FF1450B2EC15F0156EF3CF6D
:1002A00016F0152AD8B0162A15C0E5FF16C0F4FFBF
:1002B0000AC0E9FF0BC0F3FF145017EC16F074D01E
:1002C00011C0E9FF12C0F3FF1350B2EC15F0116E2C
:1002D000F3CF12F0060E1126D8B0122A1250800F5A
:1002E000F36E1050800FF35C02E10F50115C03E3DA
:1002F000F36A010E97D000C0E9FF01C0F3FF02507E
:10030000DCEC15F00A6E0A50061830E10050010FBF
:10031000066E000E01200A6E000E02200B6E06C053
:10032000E9FF0AC0F3FF0B50B2EC15F0116EF3CFEA
:1003300012F00F5011261050122211C0E5FF12C00A
:10034000F4FF06C0E9FF0AC0F3FF0B5017EC16F0EC
:10035000000EE56E000EF46E07C0E9FF08C0F3FF63
:10036000095017EC16F0F36A020E5CD0070E002657
:10037000000E0122000E022200C0E9FF01C0F3FFBF
:100380000250B2EC15F0066EF3CF0AF0062AD8B090
:100390000A2A06C0E5FF0AC0F4FF00C0E9FF01C059
:1003A000F3FF025017EC16F00F50FF0F006EFF0E18
:1003B0001020016E0150800F800F02E1010E005CE1
:1003C00024E300500C24026E01500D20066EE86AF2
:1003D00001BEE8680E200A6E02C0E9FF06C0F3FF06
:1003E0000A50DCEC15F0026E0250E56E0550E56E29
:1003F0000450E56E0350E56E6EEC0EF0040EE1263F
:10040000FF0E0026D8A00106D5D7000EE56E000E1F
:10041000F46E07C0E9FF08C0F3FF095017EC16F0AF
:10042000F36AE86AE4CF16F0E4CF15F0E4CF14F0F5
:10043000E4CF13F0E4CF12F0E4CF11F0E4CF10F0EA
:10044000E4CF0FF0E4CF0EF0E4CF0DF0E4CF0CF0EA
:10045000E4CF0BF0E4CF0AF0E4CF09F0E4CF08F0EA
:10046000E4CF07F0E4CF06F0E4CF05F0E4CF04F0EA
:10047000E4CF03F0E4CF02F0E4CF01F0E4CF00F0EA
:10048000E4CFD9FF1200D9CFE5FFE1CFD9FF00C0FB
:10049000E5FF01C0E5FF02C0E5FF03C0E5FF04C0C2
:1004A000E5FF05C0E5FF06C0E5FF07C0E5FF08C0A2
:1004B000E5FF09C0E5FF0AC0E5FF0BC0E5FF0CC082
:1004C000E5FF0DC0E5FF0EC0E5FF0FC0E5FF10C062
:1004D000E5FF11C0E5FF12C0E5FF13C0E5FF14C042
:1004E000E5FF020EDBCF00F0030EDBCF01F0040EC0
:1004F000DBCF02F0050EDBCF03F0060EDBCF04F0FE
:10050000070EDBCF05F0080EDBCF06F0090EDBCFC0
:1005100007F00A0EDBCF08F00B0EDBCF09F00C0E54
:10052000DBCF0AF00D0EDBCF0BF00801836B60AE62
:1005300029D0A49074AE13D009C0E9FF0AC0F3FF1C
:100540000B50DCEC15F00C6E0C860CC0E5FF09C0FE
:10055000E9FF0AC0F3FF0B5023EC16F0749E0C6AFF
:1005600060B00C2A0C50010BF46E08018351FE0B95
:10057000F4100801836F0F0E0D6E600E0C6E800E6E
:100580000E6E40D00F0150AF3BD0A49274AC13D08C
:1005900009C0E9FF0AC0F3FF0B50DCEC15F00F6E49
:1005A0000F860FC0E5FF09C0E9FF0AC0F3FF0B503B
:1005B00023EC16F0749C070E0F0150150F6E0F50B0
:1005C0000801836F83C8E8FF020E0F5C12E209C0C6
:1005D000E9FF0AC0F3FF0B50DCEC15F00F6E0F8E35
:1005E0000FC0E5FF09C0E9FF0AC0F3FF0B5023EC81
:1005F00016F00F0E0D6E500E0C6E800E0E6E02D0A9
:10060000E86AFFD00CC00FF00DC010F00EC011F062
:10061000000EE56E09C0E9FF0AC0F3FF0B5023ECA2
:1006200016F00C50050F126E000E0D20136E000E0A
:100630000E20146E12C0E9FF13C0F3FF1450DCEC5F
:1006400015F0126E12500801846F84C8E8FF0F0E77
:10065000121612C0E5FF06C0E9FF07C0F3FF0850FD
:1006600023EC16F0080184AD12D009C0E9FF0AC0DE
:10067000F3FF0B50DCEC15F0126E128C12C0E5FF8C
:1006800009C0E9FF0AC0F3FF0B5023EC16F00C5031
:10069000020F126E000E0D20136E000E0E20146E4F
:1006A00012C0E9FF13C0F3FF1450DCEC15F0126E1A
:1006B00012500801846F080184A716D009C0E9FF11
:1006C0000AC0F3FF0B50DCEC15F0126E128A12C058
:1006D000E5FF09C0E9FF0AC0F3FF0B5023EC16F059
:1006E000010E0801846F02D00801846B0C50010FC9
:1006F000126E000E0D20136E000E0E20146E0801F7
:100700008451E56E0250E56E0150E56E0050E56ED5
:100710001450E56E1350E56E1250E56E85EC0AF04C
:10072000070EE126060E0C26000E0D22000E0E22EC
:1007300006C0E9FF07C0F3FF0850DCEC15F0066EB9
:1007400006500801846F0CC000F00DC001F00EC00F
:1007500002F0066A06C007F0086A06BE086884C888
:100760000CF00D6A0850800FF36E0D50800FF35C93
:1007700002E10C50075C1DE200C0E9FF01C0F3FF7D
:100780000250DCEC15F0076E002AD8B0012AD8B070
:10079000022A07C0E5FF03C0E9FF04C0F3FF0550CC
:1007A00023EC16F0032AD8B0042AD8B0052A062A6A
:1007B000D1D7A4AE13D009C0E9FF0AC0F3FF0B5094
:1007C000DCEC15F0006E008800C0E5FF09C0E9FF11
:1007D0000AC0F3FF0B5023EC16F0A49E0FC0E9FFF4
:1007E00010C0F3FF1150DCEC15F0006E009E00C04D
:1007F000E5FF0FC0E9FF10C0F3FF115023EC16F026
:10080000010EE4CF14F0E4CF13F0E4CF12F0E4CF04
:1008100011F0E4CF10F0E4CF0FF0E4CF0EF0E4CF0E
:100820000DF0E4CF0CF0E4CF0BF0E4CF0AF0E4CF0E
:1008300009F0E4CF08F0E4CF07F0E4CF06F0E4CF0E
:1008400005F0E4CF04F0E4CF03F0E4CF02F0E4CF0E
:1008500001F0E4CF00F0E4CFD9FF1200D9CFE5FFDB
:10086000E1CFD9FF00C0E5FF01C0E5FF02C0E5FF11
:1008700003C0E5FF04C0E5FF05C0E5FF06C0E5FFD6
:1008800007C0E5FF08C0E5FF09C0E5FF0AC0E5FFB6
:100890000BC0E5FF0CC0E5FF0DC0E5FF0EC0E5FF96
:1008A0000FC0E5FF10C0E5FF11C0E5FF12C0E5FF76
:1008B00013C0E5FF14C0E5FF020EDBCF00F0030E0E
:1008C000DBCF01F0040EDBCF02F0050EDBCF03F02F
:1008D000060EDBCF04F0070EDBCF05F00050440F0F
:1008E000066E000E0120076E000E0220086E06C084
:1008F000E9FF07C0F3FF08507EEC15F0096EF3CF57
:100900000AF0F4CF0BF00050340F0C6E000E0120F3
:100910000D6E000E02200E6E09500C1806E10A50F2
:100920000D1803E10B500E1801E09FD00050410F4D
:100930000C6E000E01200D6E000E02200E6E0CC01B
:10094000E9FF0DC0F3FF0E507EEC15F00C6EF3CFF7
:100950000DF0F4CF0EF00C50001807E10D50011807
:1009600004E10E50021801E124D10950040F0C6E6D
:10097000000E0A200D6E000E0B200E6E0350040FA9
:100980000F6E000E0420106E000E0520116E000E7A
:10099000E56E080EE56E1150E56E1050E56E0F50D5
:1009A000E56E0E50E56E0D50E56E0C50E56E54ECA4
:1009B00013F0080EE12606C0E9FF07C0F3FF085058
:1009C0007EEC15F00C6EF3CF0DF0F4CF0EF00C5062
:1009D0000C0F0F6E000E0D20106E000E0E20116E0B
:1009E00003500C0F126E000E0420136E000E052033
:1009F000146E12C0E9FF13C0F3FF1450DCEC15F0C5
:100A0000126E12C0E5FF0FC0E9FF10C0F3FF1150D6
:100A100023EC16F003C0E9FF04C0F3FF055023ECFC
:100A200015F00F6EF3CF10F0F4CF11F0E9CF12F004
:100A30000FC0E5FF10C0F4FF11C0F6FF12C0F7FFB2
:100A40000CC0E9FF0DC0F3FF0E50EDEC15F000C037
:100A5000E5FF01C0F4FF02C0F6FF06C0E9FF07C0D2
:100A6000F3FF0850FDEC15F0A4D0410E0026000E57
:100A70000122000E022200C0E9FF01C0F3FF025074
:100A80007EEC15F0006EF3CF01F0F4CF02F0F30E20
:100A90000026FF0E0122FF0E02220950001807E176
:100AA0000A50011804E10B50021801E182D0040E33
:100AB0000926000E0A22000E0B220350040F006EBE
:100AC000000E0420016E000E0520026E000EE56E81
:100AD000080EE56E0250E56E0150E56E0050E56EC1
:100AE0000B50E56E0A50E56E0950E56E54EC13F0BC
:100AF000080EE12606C0E9FF07C0F3FF08507EECB0
:100B000015F0006EF3CF01F0F4CF02F000500C0F9F
:100B1000096E000E01200A6E000E02200B6E0350BB
:100B20000C0F0C6E000E04200D6E000E05200E6ED4
:100B30000CC0E9FF0DC0F3FF0E50DCEC15F00C6E9D
:100B40000CC0E5FF09C0E9FF0AC0F3FF0B5023EC1E
:100B500016F003C0E9FF04C0F3FF055023EC15F0C5
:100B6000036EF3CF04F0F4CF05F0E9CF09F003C032
:100B7000E5FF04C0F4FF05C0F6FF09C0F7FF00C0A1
:100B8000E9FF01C0F3FF0250EDEC15F00D0E002659
:100B9000000E0122000E022200C0E5FF01C0F4FF9A
:100BA00002C0F6FF06C0E9FF07C0F3FF0850FDECE6
:100BB00015F0E4CF14F0E4CF13F0E4CF12F0E4CF5B
:100BC00011F0E4CF10F0E4CF0FF0E4CF0EF0E4CF5B
:100BD0000DF0E4CF0CF0E4CF0BF0E4CF0AF0E4CF5B
:100BE00009F0E4CF08F0E4CF07F0E4CF06F0E4CF5B
:100BF00005F0E4CF04F0E4CF03F0E4CF02F0E4CF5B
:100C000001F0E4CF00F0E4CFD9FF1200060E006E31
:100C1000016A000E036E600E026E800E046E0250BA
:100C20000001B06F03500001B16F04500001B26FBA
:100C3000000E036E600E026E800E046E0250000104
:100C4000B36F03500001B46F04500001B56F450E3F
:100C50000001B66F0001C56B0001C66BA2EC14F079
:100C600099EC15F0080E0001FE6F000E0001FD6FFB
:100C7000800E0001FF6FFDC002F0FEC003F0FFC058
:100C800004F0410E0226000E0322000E0422FDC0D5
:100C900005F0FEC006F0FFC007F005C0E5FF06C086
:100CA000F4FF07C0F6FF02C0E9FF03C0F3FF0450E2
:100CB000FDEC15F0FDC002F0FEC003F0FFC004F033
:100CC000440E0226000E0322000E0422FDC005F091
:100CD000FEC006F0FFC007F005C0E5FF06C0F4FF48
:100CE00007C0F6FF02C0E9FF03C0F3FF0450FDECAC
:100CF00015F0FDC002F0FEC003F0FFC004F0470E87
:100D00000226000E0322000E0422FDC005F0FEC0E4
:100D100006F0FFC007F005C0E5FF06C0F4FF07C0FE
:100D2000F6FF02C0E9FF03C0F3FF0450FDEC15F02D
:100D3000FDC002F0FEC003F0FFC004F04A0E022620
:100D4000000E0322000E0422450EE56E02C0E9FFEC
:100D500003C0F3FF045023EC16F0D08ED76AD66A96
:100D6000020ED56E9D8A9F8AA380A382A580A5824C
:100D7000A38EA38AA58AA58EF28ED584D582D5842A
:100D800000C002F001C003F0046A056A0001B0511E
:100D90000001B3190BE10001B1510001B41906E1E2
:100DA0000001B2510001B51901E147D00550800F93
:100DB000800F02E1030E045CD8B03FD0022AD8B005
:100DC000032A000E076EBC0E066E800E086E000E23
:100DD0000A6E600E096E800E0B6E0B50E56E0A50A7
:100DE000E56E0950E56E0850E56E0750E56E065059
:100DF000E56E06EC00F00001BA6FF3CFBBF0060E13
:100E0000E1260001BA51020A03E10001BB5101E0F1
:100E1000BDD7000E076EBC0E066E800E086E085021
:100E2000E56E0750E56E0650E56ED9EC13F0030E43
:100E3000E126042AD8B0052AA9D702C000F003C0D1
:100E400001F0026AABB2022A0250010A01E1AB983A
:100E5000ABB801D0AB88026A036AFDC004F0FEC0E3
:100E600005F0FFC006F0410E0426000E0522000E1C
:100E7000062204C0E9FF05C0F3FF06507EEC15F022
:100E8000046EF3CF05F0F4CF06F0FDC007F0FEC00E
:100E900008F0FFC009F0440E0726000E0822000EDD
:100EA000092207C0E9FF08C0F3FF09507EEC15F0E6
:100EB000076EF3CF08F0F4CF09F00450071807E1EC
:100EC0000550081804E10650091801E159D70350EC
:100ED000800F800F02E1030E025CD8B051D7080EDC
:100EE000056E660E046E800E066E0650E56E0550A9
:100EF000E56E0450E56E0001FF51E56E0001FE5104
:100F0000E56E0001FD51E56E37EC0DF0060EE126B1
:100F1000080E056E660E046E800E066E0650E56EB7
:100F20000550E56E0450E56E0001FF51E56E0001CD
:100F3000FE51E56E0001FD51E56E45EC10F0060E28
:100F4000E126022AD8B0032A006A016A86D7120075
:100F5000D9CFE5FFE1CFD9FF00C0E5FF01C0E5FF34
:100F600002C0E5FF03C0E5FF04C0E5FF05C0E5FFE3
:100F700006C0E5FF07C0E5FF08C0E5FF09C0E5FFC3
:100F80000AC0E5FF0BC0E5FF0CC0E5FF0DC0E5FFA3
:100F90000EC0E5FF0FC0E5FF10C0E5FF11C0E5FF83
:100FA00012C0E5FF13C0E5FF14C0E5FF15C0E5FF63
:100FB000020EDBCF00F0030EDBCF01F0040EDBCF1F
:100FC00002F0050EDBCF03F0060EDBCF04F0070EB8
:100FD000DBCF05F0080EDBCF06F0090EDBCF07F004
:100FE0000A0EDBCF08F00F0E0A6E400E096E800E5F
:100FF0000B6E095008014B6F0A5008014C6F0B50E3
:1010000008014D6F0F0E0A6E300E096E800E0B6ECA
:10101000095008014E6F0A5008014F6F0B5008012C
:10102000506F0F0E0A6E200E096E800E0B6E095067
:101030000801516F0A500801526F0B500801536F9D
:10104000096A0A6A020E095CD8B0C5D04B0E0A24A0
:101050000B6E0C6A080E0C220BC0E9FF0CC0EAFFF5
:10106000EECF0BF0EECF0CF0EFCF0DF00BC00EF08B
:101070000CC00FF00DC010F00BC0E9FF0CC0F3FF67
:101080000D50DCEC15F0116E11B6A1D0FC0E11164E
:1010900011C0E5FF0BC0E9FF0CC0F3FF0D5023ECBE
:1010A00016F00BC0E9FF0CC0F3FF0D50DCEC15F09F
:1010B000116E030E0814126E1250111211C0E5FFCA
:1010C0000BC0E9FF0CC0F3FF0D5023EC16F008AC89
:1010D00004D0400E0710116E02D007C011F00B5063
:1010E000050F126E000E0C20136E000E0D20146EF4
:1010F00011C0E5FF12C0E9FF13C0F3FF145023EC49
:1011000016F008AA03D0010E116E01D0116A0B501F
:10111000010F126E000E0C20136E000E0D20146EC7
:101120001150E56E0350E56E0250E56E0150E56E1C
:101130000050E56E1450E56E1350E56E1250E56EEA
:10114000EDEC0BF0080EE126060E0B26000E0C222D
:10115000000E0D2204C011F005C012F006C013F0FD
:10116000146A0750145C1DE211C0E9FF12C0F3FFBE
:101170001350DCEC15F0156E112AD8B0122AD8B035
:10118000132A15C0E5FF0BC0E9FF0CC0F3FF0D509B
:1011900023EC16F00B2AD8B00C2AD8B00D2A142A4A
:1011A000E0D70EC0E9FF0FC0F3FF1050DCEC15F0E4
:1011B0000B6E0BB40AD00B860BC0E5FF0EC0E9FF27
:1011C0000FC0F3FF105023EC16F0010E05D0030EF4
:1011D0000A26092A37D7E86AE4CF15F0E4CF14F0DD
:1011E000E4CF13F0E4CF12F0E4CF11F0E4CF10F02D
:1011F000E4CF0FF0E4CF0EF0E4CF0DF0E4CF0CF02D
:10120000E4CF0BF0E4CF0AF0E4CF09F0E4CF08F02C
:10121000E4CF07F0E4CF06F0E4CF05F0E4CF04F02C
:10122000E4CF03F0E4CF02F0E4CF01F0E4CF00F02C
:10123000E4CFD9FF1200E8CFE5FFD8CFE5FFE0CF3C
:10124000E5FFF3CFE5FFF4CFE5FFE9CFE5FFEACF18
:10125000E5FFFACFE5FFFBCFE5FFD9CFE5FFE1CF13
:10126000D9FF00C0E5FF01C0E5FF02C0E5FF03C0F4
:10127000E5FF04C0E5FF05C0E5FF06C0E5FF07C0C8
:10128000E5FF08C0E5FF09C0E5FF0AC0E5FF0BC0A8
:10129000E5FF006A9EBA002A0050010A2DE1000114
:1012A000E32B02E30001E42B006A016A3CEC16F038
:1012B000026E025020E00150800F800F02E1140EF8
:1012C000005C19E2000E036E600E026E800E046E6A
:1012D000C8EC15F0056E0550E56E0450E56E035040
:1012E000E56E0250E56E5DEC0FF0040EE126002A7B
:1012F000D8B0012ADBD79E9A006AA4B0002A005019
:10130000010A01E0D5D0006A60BE002A0050010A3F
:1013100001E053D0D5BE03D0D76AD66AD58E000E71
:10132000016EE70E006E800E026E000E046EEB0E74
:10133000036E800E056E000E076EF30E066E800EB5
:10134000086E080E0A6E820E096E800E0B6E0B5030
:10135000E56E0A50E56E0950E56E0850E56E0750DF
:10136000E56E0650E56E0550E56E0450E56E0350DF
:10137000E56E0250E56E0150E56E0050E56E43ECFF
:1013800002F00C0EE126000E016EE70E006E800EDC
:10139000026E0250E56E0150E56E0050E56E0001F0
:1013A000FF51E56E0001FE51E56E0001FD51E56E55
:1013B0002EEC04F0060EE126609E0001E751110AB2
:1013C0000AE10001E851010A06E10001E95103E1E7
:1013D0000001EA5101E06BD00001BF51006E016ACB
:1013E00000500001F56F0001C051006E016A00BE9F
:1013F0000168016A00500001F66F0001C151006EE2
:10140000016A00500001F76F0001C251006E016ACD
:1014100000BE0168016A00500001F86F0001C3516D
:10142000006E016A00500001F96F0001C451006EA6
:10143000016A00BE0168016A00500001FA6F0001F4
:10144000BD51006E016A00500001FB6F0001BE51EA
:10145000006E016A00BE0168016A00500001FC6F65
:10146000080E0801816F000E016EF50E006E800EF1
:10147000026E000EE56E08018151E56E0250E56EC8
:101480000150E56E0050E56E08017651E56E0801E9
:101490007551E56E08017451E56E08017351E56EF2
:1014A000A8EC07F0006E090EE1260050DCE0A490E5
:1014B000E4CF0BF0E4CF0AF0E4CF09F0E4CF08F07A
:1014C000E4CF07F0E4CF06F0E4CF05F0E4CF04F07A
:1014D000E4CF03F0E4CF02F0E4CF01F0E4CF00F07A
:1014E000E4CFD9FFE4CFFBFFE4CFFAFFE4CFEAFF7C
:1014F000E4CFE9FFE4CFF4FFE4CFF3FFE4CFE0FF74
:10150000E4CFD8FFE4CFE8FF1000D9CFE5FFE1CF6B
:10151000D9FF00C0E5FF01C0E5FF02C0E5FF03C041
:10152000E5FF04C0E5FF05C0E5FF06C0E5FF07C015
:10153000E5FF08C0E5FF09C0E5FF0AC0E5FF0BC0F5
:10154000E5FF0CC0E5FF0DC0E5FF020EDBCF00F0AC
:10155000030EDBCF01F0040EDBCF02F0050EDBCF74
:1015600003F0060EDBCF04F0070EDBCF05F0080E0C
:10157000DBCF06F00650D8A46CD000C0E9FF01C054
:10158000F3FF0250DCEC15F0066E0638E840F80B6D
:10159000076E07C0E5FF03C0E9FF04C0F3FF055075
:1015A00023EC16F00350010F086E000E0420096EA4
:1015B000000E05200A6E0638E840070B066E06C0CE
:1015C000E5FF08C0E9FF09C0F3FF0A5023EC16F05D
:1015D000002AD8B0012AD8B0022A00C0E9FF01C011
:1015E000F3FF0250DCEC15F0066E0638E840070BFE
:1015F000066E0650071207C0E5FF03C0E9FF04C0EE
:10160000F3FF055023EC16F00350020F066E000E98
:101610000420076E000E0520086E000EE56E06C061
:10162000E9FF07C0F3FF085023EC16F00350030F47
:10163000066E000E0420076E000E0520086E000ED8
:10164000E56E06C0E9FF07C0F3FF085023EC16F073
:10165000A5D00350020F066E000E0420076E000E88
:101660000520086E00C0E9FF01C0F3FF0250DCEC6A
:1016700015F0096E0938E844E00B0A6E0AC0E5FF70
:1016800006C0E9FF07C0F3FF085023EC16F0035033
:10169000030F0B6E000E04200C6E000E05200D6E65
:1016A0000938E8441F0B096E09C0E5FF0BC0E9FFCC
:1016B0000CC0F3FF0D5023EC16F0002AD8B0012A1D
:1016C000D8B0022A06C0E9FF07C0F3FF0850DCECDF
:1016D00015F0E86E00C0E9FF01C0F3FF0250DCEC3A
:1016E00015F0096E030E09140B6E0B500A120AC096
:1016F000E5FF06C0E9FF07C0F3FF085023EC16F032
:1017000006C0E9FF07C0F3FF0850DCEC15F0E86EF7
:10171000E00E09160938E8441F0B096E09500A1239
:101720000AC0E5FF06C0E9FF07C0F3FF085023EC3D
:1017300016F0002AD8B0012AD8B0022A0350010FAF
:10174000066E000E0420076E000E0520086E00C015
:10175000E9FF01C0F3FF0250DCEC15F0096E09C08F
:10176000E5FF06C0E9FF07C0F3FF085023EC16F0C1
:10177000002AD8B0012AD8B0022A00C0E9FF01C06F
:10178000F3FF0250DCEC15F0006E00C0E5FF03C073
:10179000E9FF04C0F3FF055023EC16F0E4CF0DF091
:1017A000E4CF0CF0E4CF0BF0E4CF0AF0E4CF09F083
:1017B000E4CF08F0E4CF07F0E4CF06F0E4CF05F083
:1017C000E4CF04F0E4CF03F0E4CF02F0E4CF01F083
:1017D000E4CF00F0E4CFD9FF1200D9CFE5FFE1CF8D
:1017E000D9FF00C0E5FF01C0E5FF02C0E5FF03C06F
:1017F000E5FF04C0E5FF05C0E5FF06C0E5FF07C043
:10180000E5FF08C0E5FF09C0E5FF0AC0E5FF020EDD
:10181000DBCF00F0030EDBCF01F0040EDBCF02F0D4
:10182000050EDBCF7BF8060EDBCF7CF8070EDBCF97
:101830007DF8080EDBCF7EF8090EDBCF03F0080E33
:10184000056E7B0E046E800E066E0350D8A450D039
:1018500004C0E9FF05C0F3FF0650DCEC15F0036E91
:101860000338E8441F0B076E07C0E5FF00C0E9FF1F
:1018700001C0F3FF025023EC16F000C0E9FF01C0E5
:10188000F3FF0250DCEC15F0076E0450010F086EF8
:10189000000E0520096E000E06200A6E08C0E9FF42
:1018A00009C0F3FF0A50DCEC15F0086E0838E84474
:1018B000E00B096E0950071207C0E5FF00C0E9FF01
:1018C00001C0F3FF025023EC16F0002AD8B0012A21
:1018D000D8B0022A0338E844E00B076E07C0E5FFE2
:1018E00000C0E9FF01C0F3FF025023EC16F0A6D0C0
:1018F0000450020F036E000E0520076E000E062036
:10190000086E03C0E9FF07C0F3FF0850DCEC15F0D8
:10191000036E0338E840070B076E07C0E5FF00C001
:10192000E9FF01C0F3FF025023EC16F000C0E9FF0D
:1019300001C0F3FF0250DCEC15F0076E0450030FFA
:10194000086E000E0520096E000E06200A6E08C003
:10195000E9FF09C0F3FF0A50DCEC15F0086E083807
:10196000E840F80B096E0950071207C0E5FF00C0F8
:10197000E9FF01C0F3FF025023EC16F0002AD8B0B3
:10198000012AD8B0022A0338E840F80B076EE00EAF
:10199000071607C0E5FF00C0E9FF01C0F3FF0250D2
:1019A00023EC16F0078607C0E5FF00C0E9FF01C081
:1019B000F3FF025023EC16F0030E03160350071238
:1019C00007C0E5FF00C0E9FF01C0F3FF025023ECB0
:1019D00016F0002AD8B0012AD8B0022A0450010F0C
:1019E000036E000E0520076E000E0620086E03C071
:1019F000E9FF07C0F3FF0850DCEC15F0036E03C0ED
:101A0000E5FF00C0E9FF01C0F3FF025023EC16F030
:101A1000002AD8B0012AD8B0022A04C0E9FF05C0C4
:101A2000F3FF0650DCEC15F0046E04C0E5FF00C0C7
:101A3000E9FF01C0F3FF025023EC16F0E4CF0AF0F7
:101A4000E4CF09F0E4CF08F0E4CF07F0E4CF06F0EC
:101A5000E4CF05F0E4CF04F0E4CF03F0E4CF02F0EC
:101A6000E4CF01F0E4CF00F0E4CFD9FF1200D9CFEA
:101A7000E5FFE1CFD9FF00C0E5FF01C0E5FF02C0EF
:101A8000E5FF03C0E5FF04C0E5FF05C0E5FF06C0B4
:101A9000E5FF07C0E5FF08C0E5FF09C0E5FF0AC094
:101AA000E5FF0BC0E5FF0CC0E5FF0DC0E5FF0EC074
:101AB000E5FF0FC0E5FF10C0E5FF11C0E5FF020E16
:101AC000DBCF00F0030EDBCF01F0040EDBCF02F022
:101AD000050EDBCF03F0060EDBCF04F0070EDBCFE5
:101AE00005F00050410F066E000E0120076E000E3B
:101AF0000220086E06C0E9FF07C0F3FF08507EEC25
:101B000015F0096EF3CF0AF0F4CF0BF00050440F3C
:101B10000C6E000E01200D6E000E02200E6E0CC029
:101B2000E9FF0DC0F3FF0E507EEC15F00C6EF3CF05
:101B30000DF0F4CF0EF009500C1807E10A500D1803
:101B400004E10B500E1801E1A2D00350040F0C6EFB
:101B5000000E04200D6E000E05200E6E040E0926E8
:101B6000000E0A22000E0B22000EE56E080EE56E36
:101B70000B50E56E0A50E56E0950E56E0E50E56EAD
:101B80000D50E56E0C50E56E54EC13F0080EE12696
:101B900003500C0F096E000E04200A6E000E052083
:101BA0000B6E06C0E9FF07C0F3FF08507EEC15F08E
:101BB0000C6EF3CF0DF0F4CF0EF00C500C0F0F6E37
:101BC000000E0D20106E000E0E20116E0FC0E9FFEA
:101BD00010C0F3FF1150DCEC15F00F6E0FC0E5FFE5
:101BE00009C0E9FF0AC0F3FF0B5023EC16F00CC04C
:101BF000E9FF0DC0F3FF0E5023EC15F0096EF3CF93
:101C00000AF0F4CF0BF0E9CF0FF009C0E5FF0AC0EE
:101C1000F4FF0BC0F6FF0FC0F7FF03C0E9FF04C0DD
:101C2000F3FF0550EDEC15F00050340F036E000E7D
:101C30000120046E000E0220056E0C50031806E110
:101C40000D50041803E10E50051814E00D0E0C267B
:101C5000000E0D22000E0E220CC0E5FF0DC0F4FF99
:101C60000EC0F6FF06C0E9FF07C0F3FF0850FDEC09
:101C700015F00DD000C0E5FF01C0F4FF02C0F6FF73
:101C800006C0E9FF07C0F3FF0850FDEC15F0E4CFF4
:101C900011F0E4CF10F0E4CF0FF0E4CF0EF0E4CF7A
:101CA0000DF0E4CF0CF0E4CF0BF0E4CF0AF0E4CF7A
:101CB00009F0E4CF08F0E4CF07F0E4CF06F0E4CF7A
:101CC00005F0E4CF04F0E4CF03F0E4CF02F0E4CF7A
:101CD00001F0E4CF00F0E4CFD9FF1200D9CFE5FF47
:101CE000E1CFD9FF00C0E5FF01C0E5FF02C0E5FF7D
:101CF00003C0E5FF04C0E5FF05C0E5FF06C0E5FF42
:101D000007C0E5FF08C0E5FF09C0E5FF0AC0E5FF21
:101D10000BC0E5FF0CC0E5FF0DC0E5FF0EC0E5FF01
:101D20000FC0E5FF020EDBCF00F0030EDBCF01F0AA
:101D3000040EDBCF02F0050EDBCF03F00050500F96
:101D4000046E000E0120056E000E0220066E04C017
:101D5000E9FF05C0F3FF06507EEC15F0076EF3CFE8
:101D600008F0F4CF09F00750001806E108500118F8
:101D700003E10950021801E042D00050530F0A6EEF
:101D8000000E01200B6E000E02200C6E0AC0E9FF4F
:101D90000BC0F3FF0C507EEC15F00A6EF3CF0BF086
:101DA000F4CF0CF000504F0F0D6E000E01200E6EA0
:101DB000000E02200F6E0A500D1806E10B500E188F
:101DC00003E10C500F1801E003D0F36AE86A52D027
:101DD0000DC0E5FF0EC0F4FF0FC0F6FF04C0E9FF21
:101DE00005C0F3FF0650FDEC15F003C0E5FF0DC084
:101DF000E9FF0EC0F3FF0F5023EC16F03BD0530E5B
:101E00000026000E0122000E022200C0E9FF01C0E0
:101E1000F3FF02507EEC15F0006EF3CF01F0F4CF2B
:101E200002F0FF0E0726FF0E0822FF0E09220050C7
:101E3000071806E10150081803E10250091801E0F3
:101E400003D0F36AE86A16D007C0E5FF08C0F4FFC4
:101E500009C0F6FF04C0E9FF05C0F3FF0650FDEC22
:101E600015F003C0E5FF07C0E9FF08C0F3FF095004
:101E700023EC16F0E4CF0FF0E4CF0EF0E4CF0DF03A
:101E8000E4CF0CF0E4CF0BF0E4CF0AF0E4CF09F09C
:101E9000E4CF08F0E4CF07F0E4CF06F0E4CF05F09C
:101EA000E4CF04F0E4CF03F0E4CF02F0E4CF01F09C
:101EB000E4CF00F0E4CFD9FF1200D9CFE5FFE1CFA6
:101EC000D9FF00C0E5FF01C0E5FF02C0E5FF03C088
:101ED000E5FF04C0E5FF05C0E5FF06C0E5FF07C05C
:101EE000E5FF08C0E5FF09C0E5FF0AC0E5FF0BC03C
:101EF000E5FF0CC0E5FF020EDBCF00F0030EDBCFE9
:101F000001F0040EDBCF02F0050EDBCF03F0005032
:101F1000530F046E000E0120056E000E0220066EA7
:101F200004C0E9FF05C0F3FF06507EEC15F0076E14
:101F3000F3CF08F0F4CF09F000504F0F0A6E000EF7
:101F400001200B6E000E02200C6E07500A1806E1ED
:101F500008500B1803E109500C1801E039D000506B
:101F6000500F0A6E000E01200B6E000E02200C6E48
:101F70000AC0E9FF0BC0F3FF0C507EEC15F00A6EAF
:101F8000F3CF0BF0F4CF0CF00A50001806E10B5021
:101F9000011803E10C50021801E003D0F36AE86A6B
:101FA00057D003C0E5FF07C0E9FF08C0F3FF0950A1
:101FB00023EC16F000C0E5FF01C0F4FF02C0F6FFFD
:101FC00004C0E9FF05C0F3FF0650FDEC15F040D05A
:101FD000500E0026000E0122000E022200C0E9FF72
:101FE00001C0F3FF02507EEC15F0006EF3CF01F05C
:101FF000F4CF02F0FF0E0026FF0E0122FF0E022298
:102000000750001806E10850011803E109500218B2
:1020100001E003D0F36AE86A1BD003C0E5FF07C004
:10202000E9FF08C0F3FF095023EC16F0072AD8B0E7
:10203000082AD8B0092A07C0E5FF08C0F4FF09C084
:10204000F6FF04C0E9FF05C0F3FF0650FDEC15F0F4
:10205000E4CF0CF0E4CF0BF0E4CF0AF0E4CF09F0CA
:10206000E4CF08F0E4CF07F0E4CF06F0E4CF05F0CA
:10207000E4CF04F0E4CF03F0E4CF02F0E4CF01F0CA
:10208000E4CF00F0E4CFD9FF1200D9CFE5FFE1CFD4
:10209000D9FF00C0E5FF01C0E5FF02C0E5FF03C0B6
:1020A000E5FF04C0E5FF05C0E5FF06C0E5FF07C08A
:1020B000E5FF08C0E5FF09C0E5FF0AC0E5FF0BC06A
:1020C000E5FF050EDBCF00F0060EDBCF01F0070EBB
:1020D000DBCF02F0AA0E036E00C004F001C005F0D1
:1020E00002C006F0AA0E2DEC16F040EC16F0076EBA
:1020F0000750FBE1076A086A0850800F800F02E171
:10210000040E075C21E207500424096E08500520E4
:102110000A6EE86A08BEE86806200B6E09C0E9FF8F
:102120000AC0F3FF0B50DCEC15F0096E09500326D2
:1021300009502DEC16F040EC16F0096E0950FBE149
:10214000072AD8B0082AD8D700500C0F046E000E0A
:102150000120056E000E0220066E04C0E9FF05C0D6
:10216000F3FF0650DCEC15F0076E07502DEC16F06F
:1021700040EC16F0076E0750FBE104C0E9FF05C014
:10218000F3FF0650DCEC15F0076E07500326040E33
:102190000026000E0122000E0222076A086A04C00F
:1021A000E9FF05C0F3FF0650DCEC15F0096E0A6A82
:1021B0000850800FF36E0A50800FF35C02E1095063
:1021C000075C21E207500024096E085001200A6EC6
:1021D000E86A08BEE86802200B6E09C0E9FF0AC081
:1021E000F3FF0B50DCEC15F0096E09500326095083
:1021F0002DEC16F040EC16F0096E0950FBE1072AB1
:10220000D8B0082ACCD703502DEC16F0E4CF0BF051
:10221000E4CF0AF0E4CF09F0E4CF08F0E4CF07F010
:10222000E4CF06F0E4CF05F0E4CF04F0E4CF03F010
:10223000E4CF02F0E4CF01F0E4CF00F0E4CFD9FF27
:102240001200D9CFE5FFE1CFD9FF00C0E5FF01C003
:10225000E5FF02C0E5FF03C0E5FF04C0E5FF05C0E0
:10226000E5FF06C0E5FF07C0E5FF08C0E5FF09C0C0
:10227000E5FF0AC0E5FF0BC0E5FF0CC0E5FF0DC0A0
:10228000E5FF0EC0E5FF0FC0E5FF10C0E5FF020E41
:10229000DBCF00F0030EDBCF01F0040EDBCF02F04A
:1022A000036A046A0050410F056E000E0120066E9D
:1022B000000E0220076E05C0E9FF06C0F3FF0750BD
:1022C0007EEC15F0056EF3CF06F0F4CF07F000506A
:1022D000440F086E000E0120096E000E02200A6EE7
:1022E00008C0E9FF09C0F3FF0A507EEC15F0086E44
:1022F000F3CF09F0F4CF0AF00550081806E10650B4
:10230000091803E107500A1801E003D0F36AE86AEC
:1023100049D00050340F0B6E000E01200C6E000EE1
:1023200002200D6E0550081806E10650091803E159
:1023300007500A1834E005500C0F0E6E000E0620F0
:102340000F6E000E0720106E0EC0E9FF0FC0F3FFE6
:102350001050DCEC15F00E6E0F6A03500E26045080
:102360000F220E50050F036E000E0F20046E055055
:102370000B1806E106500C1803E107500D1801E098
:1023800007D000C005F001C006F002C007F0CAD7B0
:102390000D0E0526000E0622000E0722C3D704C02C
:1023A000F3FF0350E4CF10F0E4CF0FF0E4CF0EF0D2
:1023B000E4CF0DF0E4CF0CF0E4CF0BF0E4CF0AF063
:1023C000E4CF09F0E4CF08F0E4CF07F0E4CF06F063
:1023D000E4CF05F0E4CF04F0E4CF03F0E4CF02F063
:1023E000E4CF01F0E4CF00F0E4CFD9FF1200D9CF61
:1023F000E5FFE1CFD9FF00C0E5FF01C0E5FF02C066
:10240000E5FF03C0E5FF04C0E5FF05C0E5FF06C02A
:10241000E5FF07C0E5FF08C0E5FF09C0E5FF0AC00A
:10242000E5FF0BC0E5FF0CC0E5FF020EDBCF00F0BF
:10243000030EDBCF01F0040EDBCF02F00050500F93
:10244000036E000E0120046E000E0220056E03C014
:10245000E9FF04C0F3FF05507EEC15F0066EF3CFE4
:1024600007F0F4CF08F00050530F096E000E012062
:102470000A6E000E02200B6E09C0E9FF0AC0F3FFCE
:102480000B507EEC15F0096EF3CF0AF0F4CF0BF091
:102490000650091806E107500A1803E108500B1806
:1024A00001E002D0E86A3BD006C0E9FF07C0F3FFB5
:1024B0000850DCEC15F0096E00504F0F0A6E000E4C
:1024C00001200B6E000E02200C6E06500A1806E169
:1024D00007500B1803E108500C1813E0062AD8B077
:1024E000072AD8B0082A06C0E5FF07C0F4FF08C0D5
:1024F000F6FF03C0E9FF04C0F3FF0550FDEC15F043
:102500000DD000C0E5FF01C0F4FF02C0F6FF03C01C
:10251000E9FF04C0F3FF0550FDEC15F00950E4CFCE
:102520000CF0E4CF0BF0E4CF0AF0E4CF09F0E4CFF5
:1025300008F0E4CF07F0E4CF06F0E4CF05F0E4CFF5
:1025400004F0E4CF03F0E4CF02F0E4CF01F0E4CFF5
:1025500000F0E4CFD9FF1200D9CFE5FFE1CFD9FFDA
:1025600000C0E5FF01C0E5FF02C0E5FF03C0E5FFD5
:1025700004C0E5FF05C0E5FF06C0E5FF07C0E5FFB5
:1025800008C0E5FF020EDBCF00F0030EDBCF01F049
:10259000040EDBCF02F00050530F036E000E01203B
:1025A000046E000E0220056E03C0E9FF04C0F3FFB5
:1025B00005507EEC15F0036EF3CF04F0F4CF05F078
:1025C00000504F0F066E000E0120076E000E022015
:1025D000086E0350061806E10450071803E1055081
:1025E000081801E025D00050500F066E000E0120A3
:1025F000076E000E0220086E06C0E9FF07C0F3FF59
:1026000008507EEC15F0066EF3CF07F0F4CF08F01B
:102610000650001806E10750011803E1085002189F
:1026200001E003D0F36A010E2AD0F36AE86A27D0EA
:10263000500E0026000E0122000E022200C0E9FF0B
:1026400001C0F3FF02507EEC15F0006EF3CF01F0F5
:10265000F4CF02F0FF0E0026FF0E0122FF0E022231
:102660000350001806E10450011803E10550021858
:1026700001E003D0F36A010E02D0F36AE86AE4CF06
:1026800008F0E4CF07F0E4CF06F0E4CF05F0E4CFA4
:1026900004F0E4CF03F0E4CF02F0E4CF01F0E4CFA4
:1026A00000F0E4CFD9FF1200D9CFE5FFE1CFD9FF89
:1026B00000C0E5FF01C0E5FF02C0E5FF03C0E5FF84
:1026C00004C0E5FF05C0E5FF06C0E5FF07C0E5FF64
:1026D00008C0E5FF09C0E5FF0AC0E5FF0BC0E5FF44
:1026E0000CC0E5FF020EDBCF00F0030EDBCF01F0E4
:1026F000040EDBCF02F0050EDBCF03F0060EDBCFBE
:1027000004F0070EDBCF05F0080EDBCF06F0090E54
:10271000DBCF07F000C008F001C009F002C00AF0EA
:1027200006C00BF007C00CF0FF0E0626D8A0070667
:102730000B500C101CE003C0E9FF04C0F3FF055070
:10274000DCEC15F00B6E032AD8B0042AD8B0052AA9
:102750000BC0E5FF08C0E9FF09C0F3FF0A5023ECF6
:1027600016F0082AD8B0092AD8B00A2AD9D702C048
:10277000F4FF01C0F3FF0050E4CF0CF0E4CF0BF006
:10278000E4CF0AF0E4CF09F0E4CF08F0E4CF07F09B
:10279000E4CF06F0E4CF05F0E4CF04F0E4CF03F09B
:1027A000E4CF02F0E4CF01F0E4CF00F0E4CFD9FFB2
:1027B0001200D9CFE5FFE1CFD9FF00C0E5FF01C08E
:1027C000E5FF02C0E5FF03C0E5FF04C0E5FF05C06B
:1027D000E5FF020EDBCF00F0030EDBCF01F0040EAD
:1027E000DBCF02F0110E0026000E0122000E0222A5
:1027F0000050010F036E000E0120046E000E022037
:10280000056E03C0E9FF04C0F3FF055023EC15F08B
:102810000801776FF3CF78F8F4CF79F8E9CF7AF839
:102820000050050F036E000E0120046E000E022002
:10283000056E03C0E9FF04C0F3FF0550DCEC15F0A2
:10284000036E046A060E0026000E0122000E02220C
:102850000350056E000EE56E0550E56E0250E56E04
:102860000150E56E0050E56E08017A51E56E0801F1
:102870007951E56E08017851E56E08017751E56EF2
:10288000A8EC07F0056E090EE1260550E1E0E4CF63
:1028900005F0E4CF04F0E4CF03F0E4CF02F0E4CF9E
:1028A00001F0E4CF00F0E4CFD9FF12006A0EF66E1B
:1028B0002C0EF76E000EF86E0900F550056E09003B
:1028C000F550066E055002E106503BE00900F55058
:1028D000006E0900F550016E0900F550026E090006
:1028E0000900F550E96E0900F550EA6E090009008B
:1028F0000900F550036E0900F550046E0900090047
:10290000F6CF07F0F7CF08F0F8CF09F000C0F6FFD8
:1029100001C0F7FF02C0F8FF035002E1045007E0D6
:102920000900F550EE6E0306F8E20406F9D707C079
:10293000F6FF08C0F7FF09C0F8FF0506C4E2060667
:10294000C5D71200D9CFE5FFE1CFD9FF800EE56EE4
:1029500062EC15F0E12A010E706EAE0E716E050E7E
:10296000726E200E736E779E779C606A0F01506BBB
:102970000F01006B0F01016B0F01046B0F01056B61
:102980000F01086B0F01096B0F010C6B0F010D6B31
:102990000F01106B0F01116B0F01146B0F01156B01
:1029A0000F01186B0F01196B0F0119970F011C6BA9
:1029B0000F011D6B0F011D97000EE56E62EC15F007
:1029C000E12AE4CFD9FF1200D9CFE5FFE1CFD9FF4B
:1029D00000C0E5FF01C0E5FF02C0E5FF006E020E8A
:1029E000DBCF01F0030EDBCF02F0AC6AAB6A00B0C4
:1029F000AC8800A202D0AC8CAB8C00A401D0AC8E11
:102A000000A602D0AB8801D0AB8A00A802D0AC846B
:102A100001D0AC949E9800AC02D09D8A01D09D9AC2
:102A20009E9A00AE02D09D8801D09D980150AF6E55
:102A3000AC8AAB8EE4CF02F0E4CF01F0E4CF00F03B
:102A4000E4CFD9FF1200E8AE0AD0F3CFEAFFEE5090
:102A5000EECFF3FFEECFF4FFEECFE9FF1200E8BCBC
:102A600011D0E9CFF6FFF3CFF7FFF86E0900F5506C
:102A70000900F5CFF3FF0900F5CFF4FF0900F5CF0A
:102A8000E9FF12001200000000000000000000003A
:102A90000000000000000000000000000000000036
:102AA0000000000000000000000000000000000026
:102AB00000000000000064000000000000000000B2
:102AC00000000400D9CFE5FFE1CFD9FF00C0E5FF4A
:102AD00001C0E5FF020EDBCF00F01F0E6F160050A5
:102AE0006F12E00E6F14016E01500018FAE1E4CF8E
:102AF00001F0E4CF00F0E4CFD9FF1200E8AE08D037
:102B0000F3CFEAFFEE50EECFF3FFEECFF4FF12006B
:102B1000E8BC0ED0E9CFF6FFF3CFF7FFF86E09005F
:102B2000F5500900F5CFF3FF0900F5CFF4FF1200CF
:102B30001200D9CFE5FFE1CFD9FF000EE56E0A0EF6
:102B4000E56E7C0EE4EC14F0020EE1269392819285
:102B50000D0E2DEC16F0AB8ED08E9F8AF28EE4CF48
:102B6000D9FF1200E8AE06D0F3CFEAFFEE50EECF69
:102B7000F3FF1200E8BC0BD0E9CFF6FFF3CFF7FF6D
:102B8000F86E0900F5500900F5CFF3FF12001200AE
:102B9000F00E08018515856FABAC04D08591ABA014
:102BA00001D08581ABA402D008018585ABA202D0FB
:102BB00008018587AE501200E8AE04D0F3CFEAFFDB
:102BC000EE501200E8BC08D0E9CFF6FFF3CFF7FFD4
:102BD000F86E0900F55012001200E8AE0BD0F3CFEA
:102BE000EAFFE4CFEEFFF4CFEEFFF6CFEEFFF7CF34
:102BF000EEFF1200E8AC12001200E8AE09D0F3CFED
:102C0000EAFFE4CFEEFFF4CFEEFFF6CFEEFF1200C7
:102C1000E8AC1200120017EEFFF027EEFFF0F86AA2
:102C2000A68EA69C56EC14F006EC06F0FFD7E8AE94
:102C300007D0F3CFEAFFE4CFEEFFF4CFEEFF1200B0
:102C4000E8AC12001200E8AE05D0F3CFEAFFE4CF03
:102C5000EEFF1200E8AC12001200ACAC04D0AC9055
:102C6000080185B3AC80AD6E12000100862A000019
:102C7000B70000003E000000000E9EBA010F1200D7
:082C8000000EACA2010F1200CE
:020000040030CA
:0E000000FFF2FFFEFFFFBBFFFFFFFFFFFFFF52
:00000001FF
